:020000040800F2
:1020000040080020B94A0008E7270008F527000823
:1020100000000000000000000000000000000000C0
:10202000000000000000000000000000F927000888
:102030000000000000000000FB270008E92700085E
:102040003F33000800000000DF370008233A000893
:10205000B73A0008F33A0008574A0008634A0008F4
:1020600000000000E54A0008A52A0008E74A000829
:10207000E94A0008EB4A0008ED4A000800000000A9
:10208000EF4A0008F14A000800000000F34A000887
:10209000F54A0008F74A0008F94A0008FB4A000818
:1020A000FD4A0008FF4A0008014B0008034B0008E6
:1020B000054B000800B5BFF34F8F9D489D49086050
:1020C000BFF34F8F00BFFDE780B500209A4908702D
:1020D00000209A4908700020994908700020994909
:1020E000087000209849087000F03CFB9749086090
:1020F00001BD80B500F00BFC002825D100F0F0FAFE
:102100008D4908708C480078012802D100F020F930
:1021100023E089480078032802D100F07BF91CE015
:1021200085480078042802D100F0CCF915E08248F7
:102130000078022802D100F0BFF80EE000207E49AE
:10214000087000F013F808E000F00CFB7F49096804
:10215000401A652801D3FFF7ADFF01BD0120784982
:1021600008707047012075490870704710B5A7487E
:102170000078002859D12920A54908700020A449D9
:1021800048708820A24988704C20A149C8704B2013
:102190009F49087145209E49487156209C49887185
:1021A0004F209B49C8710020994908720020984926
:1021B000487200209649887200209549C872002014
:1021C000934908730020924948730020904988730E
:1021D00000208F49C87300208D49087400208C4965
:1021E000487400208A498874FF208949C874FF20F8
:1021F00087490875FF208649487588208449887575
:1022000077208349C875002004E0FF21804A121816
:102210001176401C1328F8D33120A64908703320CA
:10222000A549087000F04EFA45E0A44800F0B8FB5C
:10223000012839D1A1484078BB2802D1FFF73AFFE5
:1022400039E09E488078882826D19C48807D9B492B
:10225000CA7DFF21C9431143CA43904219D100F0FE
:102260004FFD012810D19648007800F0EBFD0400E6
:102270000A204443C148007800F0E4FD201800F033
:1022800058FD00F0B3F916E000F0B0F900F050FA94
:1022900011E000F09AF90EE0F32802D1FFF70AFFEF
:1022A000FCE700F092F906E0022802D100F08DF977
:1022B00001E000F072F910BD80B5544800780028A4
:1022C0000DD1052052490870002051494870032063
:1022D0004F49887000F054F900F0F4F926E077488F
:1022E00000F05EFB01281FD174484078BB2802D162
:1022F000FFF7E0FE1AE071488078832805D16F4827
:1023000000F0CEF900F072F910E0F92804D100F0E5
:102310006DF900F00DFA09E0F32802D1FFF7CAFECB
:10232000FCE700F052F901E000F037F901BD0000D0
:102330000400FA050CED00E0310400203304002015
:10234000320400203504002034040020EC03002077
:1023500080B52E48007800282AD10A202C49087020
:1023600000202B4948700620294988700020284900
:10237000C8700020C04300F0EFFF010E244A117125
:102380000100090C224A5171010A214A9171204928
:10239000C87100201E49087200201D4948720020A3
:1023A0001B49887200201A49C87200F08BF92BE093
:1023B000424800F0F5FA012824D140484078BB2873
:1023C00002D1FFF777FE1FE03C48807886280AD1CB
:1023D0003A4800F01CF9012802D100F007F913E097
:1023E00000F0F3F810E0F92804D100F0FFF800F055
:1023F0009FF909E0F32802D1FFF75CFEFCE700F04B
:10240000E4F801E000F0C9F801BD00003404002048
:102410005003002080B5B1480078002815D107206E
:10242000C24908700020C14948705220BF498870D5
:1024300000F0A6F800F096FF0100BC4AD171C1433C
:10244000BA48017200F03EF932E01C4800F0A8FAE8
:1024500001282BD119484078BB2802D1FFF72AFE6A
:1024600026E016488078F02809D11448C078522810
:1024700002D100F0BBF81BE000F0A7F818E0F92843
:1024800004D100F0B3F800F053F911E086280AD126
:102490000A4800F0BCF8012802D100F0A7F807E0D4
:1024A00000F093F804E000F090F801E000F075F817
:1024B00001BD00007203002073030020D002002041
:1024C000F202002080B585480078002829D10D202F
:1024D0009649087000209549487085209349887076
:1024E00000F04EF800F02EFC010E904AD171010070
:1024F000090C8E4A1172010A8C4A517201008B4AF2
:102500009172C143080E894AD0720800000C874AB4
:102510001073080A854A50738448817300F0D2F81A
:102520002AE0874800F03CFA012823D1844840780B
:10253000BB2802D1FFF7BEFD1EE081488078F0285D
:1025400009D17F48C078852802D100F04FF813E008
:1025500000F03BF810E0F92804D100F047F800F053
:10256000E7F809E0862802D100F040F804E000F026
:102570002CF801E000F011F801BD0000F30200208A
:1025800033206A49C8703120684908713020674992
:102590004871312065498871704780B500F0E2F8D4
:1025A00068490968401A65280ED300204B49087015
:1025B00065480068401C64490860634800680B284F
:1025C00002D3022000F0C2FE01BD80B55F48006862
:1025D000401C5E4908600020404908705B48006864
:1025E0000B2802D3022000F0B1FE01BD80B500200F
:1025F0005649086000205449086000203749087097
:10260000022000F09DFE01205149087001BD38B53F
:102610000400E07E227FFF21C9431143CA43904258
:102620003BD14C490978002901D100F09EFEE078A9
:102630000006217909044018617909024018A1793E
:10264000401800F0B2FB627A00231B06100A034315
:102650001206A07A00210904050C29430004801801
:102660005941E27A00231B02150E2B431202121865
:102670004B41207B002180185941627B00231302CB
:10268000002212184B41607B0021010000208018BD
:10269000594100F093FB012000E00020C0B232BDA0
:1026A00080B52D49097800290BD1C179027A12022F
:1026B0000A43417A09041143807A0006084300F076
:1026C00047FB01BD80B5194800F024F901202349DA
:1026D000087000F047F81B49086001BD3404002071
:1026E00000B51B48007801281CD10020184908704B
:1026F00018480078012804D10020164908700320EA
:1027000012E015480078012804D100201249087011
:10271000042009E012480078012801D1022003E0DA
:10272000012001E00E480078C0B200BD5003002037
:1027300000200B4908700020054908707047000010
:10274000D0020020EC030020F0030020F40300205E
:10275000350400203204002033040020340400201B
:10276000310400202A480068704780B5002009E045
:102770008100284A8918096880229205042343436E
:10278000D150401C3028F3D300F05CFE00F0D3FEA3
:1027900000F034F800F060FEFA21890000F0C8FF74
:1027A00001F01EF800210020C04301F029F80120AB
:1027B00000F025FF022000F022FF052000F01FFF9F
:1027C000032301220621144801F080F801BD80B5E1
:1027D00001F028F901BD80B501F039F901BD80B5DE
:1027E00000F074FE01BD704709480068401C0849AC
:1027F0000860704700B5FEE77047704707480068FB
:10280000032188430321014304480160704700000D
:1028100014040020002000080014004800000140BB
:102820000121C006C00E8140C3480160704780B5D9
:1028300088B0072000F0E3FE002000F0E0FE002357
:1028400001220B219020C00501F040F80023012255
:1028500008219020C00501F039F801220B219020B9
:10286000C00501F0CCF8012208219020C00501F03C
:10287000C6F8012000900323022209219020C00500
:1028800001F05DF801200090032302220A2190202C
:10289000C00501F054F8A949A94801F0EDF8A8488D
:1028A00001F004F910200190002002908020039094
:1028B0000020049000200590002006900020079042
:1028C00001A9A04801F0F8F8002001900020029032
:1028D00080200390002004900020059000200690A6
:1028E00080208001079001A9BD4801F0E5F8012191
:1028F0000A2000F085FF0A20FFF792FF01210A203D
:1029000000F07EFF0A20FFF78BFF09B000BDB5483D
:102910000078704770B5060001250220B2490870A2
:10292000002419E0305DC0B20009C0B200F09EFA88
:10293000AD490222624389184870305D0007000FDC
:1029400000F094FAA8490222624389188870002C8A
:1029500001D0305D2D18641C3078401CA042E1D2BB
:10296000E843C5B2280900F081FA9F490222624378
:10297000891848702807000F00F078FA9A49022257
:10298000624389188870032097490222624389189C
:10299000C87002204443241D200000F0D5F870BD0B
:1029A000F8B50021002200E0521CFF2A07DCB34BDF
:1029B0009B5C032BF8D111000023B04CA354FF2AD9
:1029C0006EDC00296CD04E1E00E0761E002E67D40F
:1029D000AA4A925D022AF8D10022A84B9A55891B77
:1029E000491C0839CA0701D502205AE0490800915C
:1029F0000099091F792901D3022052E00700300015
:102A0000401CC0B20100491CC9B29C4A105C9B4AE0
:102A1000515CC9B2C0B200F053F9387000983978EF
:102A2000884201D002203CE001243000C01CC0B22A
:102A30000100491CC9B2914A105C904A515CC9B26C
:102A4000C0B200F03DF9787078782418002519E0BC
:102A50003000401D022169434018C0B20100491CEA
:102A6000C9B2864A105C854A515CC9B2C0B200F056
:102A700027F9791988700098854202D278198078F0
:102A800024186D1C0098A842E2D2E043C0B200991D
:102A900079188978884201D0022002E0012000E004
:102AA0000020F2BD80B54F480078012827D1744836
:102AB00000682021084072490860002812D071483F
:102AC00000684006FBD51F480068022188431D4965
:102AD00008606D480068202101436B48016000F0E8
:102AE00085F828E0174800680821884315490860E0
:102AF0006548006880210143634801601BE011487C
:102B00000068082188430F4908600E4800680221C8
:102B100088430C4908605C48006880210901014332
:102B2000594801605848006880218900014356488F
:102B3000016000F05BF801BD00E100E081060000EB
:102B4000003801401C00024010B504000120254956
:102B5000087001220B219020C00500F050FF0122D7
:102B600008219020C00500F04AFF002003E000216A
:102B7000424A1154401CFF28F9D9444800680121F9
:102B80008843424908601648006801218843144977
:102B900008603F4804603F483F49086012483F4989
:102BA00008603A480068022101433848016037480C
:102BB0000068082101433548016039480068402118
:102BC00001433748016031480068012101432F4823
:102BD000016034480068802101433248016010BD23
:102BE0003000024030040020D000002080B50020DA
:102BF0002D490870002208219020C00500F0FFFE3A
:102C000000220B219020C00500F0F9FE002003E017
:102C100000211A4A1154401CFF28F9D91B480068AA
:102C20000121884319490860204800680121884330
:102C30001E490860802040001D4908601D481E494B
:102C400008600E481D4908601848006802210143C9
:102C500016480160154800680821014313480160C7
:102C60001248006801210143104801600D480068C6
:102C7000402101430B48016001BD0000D00100204C
:102C8000000002401C380140040002401C000240C9
:102C90002000024028380140240002402800024061
:102CA0002038014008380140300400203000024044
:102CB0003400024024380140380002403C00024009
:102CC00038B50C000021C0B200F0BCF805012000AE
:102CD000C0B200F0B7F82818C0B232BD80B500F01D
:102CE000AAFB00204F490860002000214E4A03C281
:102CF000083A00204D490860102000F027FB01BD74
:102D000080B5062805D0052803D0072801D004285F
:102D100006D146490860102000F012FB012006E0B1
:102D2000102000F013FB0020404908600020C0B2D2
:102D300002BD3F49086070473D48006870473B4806
:102D4000006870473B48006800213A4A11607047AC
:102D500039490860704780B5C0B2012807D13548AD
:102D600000688021090601433248016006E03148CD
:102D700000688021C90501432E480160FFF7F2F980
:102D800001BD00B52C480068800401D4002000E09B
:102D90000120C0B200BD80B5264800680121014372
:102DA00024480160FFF7DEF901BD1E490860704745
:102DB0001C48006870471C4803C8704780B51A4A11
:102DC00003C2083AFFF7BBFF052812D11648007866
:102DD000000707D513480068802109060143114800
:102DE00001601EE00F480068400040080D4908607F
:102DF00017E00D4803C8114A002302400B40002B86
:102E000001D1002A07D00748006880214905014305
:102E10000448016005E00348006809490140014891
:102E2000016001BD18040020E00300201C04002004
:102E300020040020240400202804002008000200B0
:102E4000FFFFFFEF00B500210100C9B230390A29A8
:102E500002D23038C0B208E00100C9B241390629B7
:102E600002D23738C0B200E0002000BD0007000FDA
:102E70000149085C70470000A84A000800B5002816
:102E800001D120207CE0C10701D5002078E0810736
:102E900001D5012074E0410701D5022070E001074F
:102EA00001D503206CE0C10601D5042068E081064D
:102EB00001D5052064E0410601D5062060E0010649
:102EC00001D507205CE0C10501D5082058E0810547
:102ED00001D5092054E0410501D50A2050E0010543
:102EE00001D50B204CE0C10401D50C2048E0810441
:102EF00001D50D2044E0410401D50E2040E001043D
:102F000001D50F203CE0C10301D5102038E081033A
:102F100001D5112034E0410301D5122030E0010336
:102F200001D513202CE0C10201D5142028E0810234
:102F300001D5152024E0410201D5162020E0010230
:102F400001D517201CE0C10101D5182018E081012E
:102F500001D5192014E0410101D51A2010E001012A
:102F600001D51B200CE0C10001D51C2008E0810028
:102F700001D51D2004E0400001D51E2000E01F20E7
:102F800000BD10B5002903D1002801D14020D5E1B2
:102F90000200D20701D50020D0E10200920701D53E
:102FA0000120CBE10200520701D50220C6E1020058
:102FB000120701D50320C1E10200D20601D5042089
:102FC000BCE10200920601D50520B7E102005206DD
:102FD00001D50620B2E10200120601D50720ADE1BD
:102FE000C20501D50820A9E1820501D50920A5E186
:102FF000420501D50A20A1E1020501D50B209DE182
:10300000C20401D50C2099E1820401D50D2095E17F
:10301000420401D50E2091E1020401D50F208DE17B
:10302000C20301D5102089E1820301D5112085E179
:10303000420301D5122081E1020301D513207DE175
:10304000C20201D5142079E1820201D5152075E173
:10305000420201D5162071E1020201D517206DE16F
:10306000C20101D5182069E1820101D5192065E16D
:10307000420101D51A2061E1020101D51B205DE169
:10308000C20001D51C2059E1820001D51D2055E167
:10309000420001D51E2051E1002801D51F204DE13D
:1030A0000022012302400B40002B01D1002A01D055
:1030B000202043E10022022302400B40002B01D1DB
:1030C000002A01D0212039E10022042302400B40D4
:1030D000002B01D1002A01D022202FE10022082359
:1030E00002400B40002B01D1002A01D0232025E112
:1030F0000022102302400B40002B01D1002A01D0F6
:1031000024201BE10022202302400B40002B01D190
:10311000002A01D0252011E10022402302400B406B
:10312000002B01D1002A01D0262007E100228023B4
:1031300002400B40002B01D1002A01D02720FDE0E6
:10314000002280235B0002400B40002B01D1002AAB
:1031500001D02820F2E0002280239B0002400B4097
:10316000002B01D1002A01D02920E7E00022802392
:10317000DB0002400B40002B01D1002A01D02A20A5
:10318000DCE0002280231B0102400B40002B01D118
:10319000002A01D02B20D1E0002280235B010240D5
:1031A0000B40002B01D1002A01D02C20C6E00022C8
:1031B00080239B0102400B40002B01D1002A01D04B
:1031C0002D20BBE000228023DB0102400B40002BBE
:1031D00001D1002A01D02E20B0E0002280231B0262
:1031E00002400B40002B01D1002A01D02F20A5E086
:1031F000002280235B0202400B40002B01D1002AF9
:1032000001D030209AE0002280239B0202400B4034
:10321000002B01D1002A01D031208FE00022802331
:10322000DB0202400B40002B01D1002A01D03220EA
:1032300084E0002280231B0302400B40002B01D1BD
:10324000002A01D0332079E0002280235B03024072
:103250000B40002B01D1002A01D034206EE0002267
:1032600080239B0302400B40002B01D1002A01D098
:10327000352063E000228023DB0302400B40002B5B
:1032800001D1002A01D0362058E0002280231B04FF
:1032900002400B40002B01D1002A01D037204DE025
:1032A000002280235B0402400B40002B01D1002A46
:1032B00001D0382042E0002280239B0402400B40D2
:1032C000002B01D1002A01D0392037E000228023D1
:1032D000DB0402400B40002B01D1002A01D03A2030
:1032E0002CE0002280231B0502400B40002B01D163
:1032F000002A01D03B2021E0002280235B05024010
:103300000B40002B01D1002A01D03C2016E0002206
:1033100080239B0502400B40002B01D1002A01D0E5
:103320003D200BE000228023DB0502400B40002BF8
:1033300001D1002A01D03E2000E03F2010BDFEE771
:1033400007490968814306480160704704490968D4
:1033500008430349086070470149096808407047FD
:10336000E80300203648006870474006400E3449A4
:103370000860704700B532480078800701D5052005
:1033800026E02F48007805210140012901D10420C1
:103390001EE02B48007825210140202901D103207F
:1033A00016E0274800787D210140082901D102203C
:1033B0000EE0234800787D210140042901D101203D
:1033C00006E01F480068002801D1002000E0062028
:1033D000C0B200BD80B50100C9B2012903D10420EB
:1033E0001749086024E00100C9B2022903D108206E
:1033F000134908601CE00100C9B2032903D1202051
:103400000F49086014E00100C9B2042903D101206A
:103410000B4908600CE0C0B2052806D108480068D6
:10342000022101430648016002E0002004490860CF
:10343000FEF794FE01BD00200149086070470000BE
:103440002C0400200348006810210143014801605A
:10345000704700000020024080B500F00DF89D4943
:103460009D4A126812091207120F895CC8409B49D5
:1034700008609A48006802BD10B5002000200020B6
:1034800000200020944800680C210140042902D04B
:10349000082902D017E0924C16E09249820C1207DC
:1034A000120F8C5C9049914A12681207120F895CC6
:1034B000C00305D58A4800F03BF96043040001E0F1
:1034C0008B48444300E0864C200010BD89480068CA
:1034D00001210143874801607F4800688649014017
:1034E0007D4801608348006884490140814801604B
:1034F00080480068824901407E4801607648006843
:103500008049014074480160784800680F21884371
:10351000764908607C480068132188437A4908602E
:103520007A4800680100C907C90F78480160002087
:1035300077490860704700B56E48006875490140DA
:103540006C4801606B4800688001FBD467480068E4
:103550000F21884365490860644800686349086032
:103560005D4800686C4901405B4801605A4800684A
:10357000A02189030143584801605E48006880210A
:10358000490401435B4801605A4800688001FBD54B
:103590006248006801210143604801604E480068AC
:1035A000F02188434C4908604B4800684A4908604C
:1035B000504800688001FBD54748006803218843D4
:1035C00045490860444800680221014342480160BF
:1035D000414800680C2101400829F9D13E480068A3
:1035E0004F4901403C4801603B4800683A49086047
:1035F0004C480068012101434A48016000BD00B504
:103600000100C9B2012907D1474800688021890219
:103610000143454801605CE00100C9B2022907D1BD
:10362000414800688021C90201433F48016050E0E1
:103630000100C9B2032907D13B4800688021090372
:1036400001433948016044E00100C9B2042907D1AF
:10365000354800688021490301433348016038E060
:103660000100C9B2052907D12F4800688021C9038C
:1036700001432D4801602CE00100C9B2062907D1A1
:103680002A4800688021C90301432848016020E0DE
:103690000100C9B2072907D1244800688021C90167
:1036A00001432248016014E00100C9B2002906D19B
:1036B0001D480068012101431B48016009E0C0B2B8
:1036C000082806D1194800688021090101431748DC
:1036D000016000BD784A000804100240CC000020C0
:1036E00000127A00884A0008984A00082C1002400C
:1036F00000093D00001002400CB8FF00FFFFF6FE7D
:10370000FFFFFBFFFFFFC0FF3010024034100240FC
:1037100008100240FFFFFFFEFFFFC2FF0020024033
:10372000FFF8FFFF0C100240141002401810024076
:103730000022030A8B420BD203098B4219D24308A1
:103740008B422ED2411A00D2014652411046704798
:10375000FF2209023FD012068B4205D31212090242
:103760008B4201D31212090203098B4219D300E0E4
:10377000090AC3098B4201D3CB01C01A5241830904
:103780008B4201D38B01C01A524143098B4201D3B2
:103790004B01C01A524103098B4201D30B01C01ADD
:1037A0005241C3088B4201D3CB00C01A5241830857
:1037B0008B4201D38B00C01A524143088B4201D384
:1037C0004B00C01A5241884200D3401A5241CFD216
:1037D00001461046704708B500F08AF908BDFEE7BB
:1037E00080B5401E2949086000210020C04300F038
:1037F00007F800202649086007202649086001BD17
:10380000F0B5020052B2002A23D5234B020052B277
:103810001207120F083A9208042462431E4C050056
:103820006DB22D072D0F083DAD0804267543645970
:10383000FF258607B60F08277E43B540AC438901B4
:10384000C9B28007800F0825684381402143995001
:103850001BE0124A03005BB29B0804246343D25866
:10386000FF238407A40F08256C43A3409A438901D2
:10387000C9B283079B0F0824634399401143074A49
:1038800040B28008042358431150F0BD14E000E01A
:1038900018E000E010E000E01CED00E000E400E0D3
:1038A00030B40368032402254D43AC40A3430360B6
:1038B000C368032402254D43AC40A343D2B2022483
:1038C00061438A401A43C26030BC704770B50468D7
:1038D000032502264E43B540AC43012502264E4344
:1038E000B540254305608468032502264E43B54054
:1038F000AC43DBB202254D43AB40234383604368B6
:1039000001248C40A343112A10D101228A401A437A
:103910004260C268032302244C43A3409A4301231C
:10392000022461438B401343C36007E04360C268D5
:103930000323022461438B409A43C26070BDF0B5FB
:10394000059C0D00EDB2082D0BDA056A0F26042741
:103950004F43BE40B54304264E43B4402C4304625B
:1039600010E0466A0F27BC460D00083D04277D4342
:103970006746AF40BE430D00083D04277D43AC4081
:10398000344344620468032502264E43B540AC43E9
:10399000022502264E43B540254305608468032571
:1039A00002264E43B540AC43DBB202254D43AB404B
:1039B00023438360436801248C40A343122A10D11F
:1039C00001228A401A434260C268032302244C4306
:1039D000A3409A430123022461438B401343C360F5
:1039E0000CE04360C268032302244C43A3409A4383
:1039F0000123022461438B401343C360F0BD00B533
:103A0000D2B2002A03D001228A40826103E001225F
:103A100010318A40826100BD026901208840104057
:103A20007047FEE700B50C480C4908600C480B498C
:103A3000086000200B4908600B480C4908600C48DE
:103A400000680028FBD10B480449086000BD094804
:103A50000249086070470000CCCC000000300040F4
:103A60005555000004300040FF0F000008300040B2
:103A70000C300040AAAA0000002202600268084B35
:103A8000134303604268074B13404360C1604168C1
:103A9000054A0A40426081682A229143816070474A
:103AA0000C800000FFCFFFFFFFB7FFFF016801227E
:103AB0000A4302607047FEE710B4026801239A438C
:103AC00002600368094A1A400B684C681C438B6803
:103AD0002343CC681C430B6923434C691C4389690D
:103AE00021431143016010BC704700BF0FC0FFFFAE
:103AF0007047FEE780B50023012200219020C00519
:103B0000FFF7E4FE0023012201219020C005FFF70A
:103B1000DDFE0023012202219020C005FFF7D6FE22
:103B20000023012203219020C005FFF7CFFE0023D0
:103B3000012204219020C005FFF7C8FE00230122C6
:103B400005219020C005FFF7C1FE00220021902032
:103B5000C005FFF754FF002201219020C005FFF7A8
:103B60004EFF002202219020C005FFF748FF0022EF
:103B700003219020C005FFF742FF0022042190207E
:103B8000C005FFF73CFF002205219020C005FFF78C
:103B900036FFFEF7E7FD7B49086000F04EFA7A48F1
:103BA0000078012101437848017001BD7749087010
:103BB000704780B50120FFF7CFFB002805D03F20DC
:103BC00000F0EAF800F039FADBE00220FFF7C4FB6E
:103BD000002804D11020FFF7BFFB002805D03F20AC
:103BE00000F001FA00F029FACBE0684800780128DB
:103BF00005D1122000F0D0F800F01FFAC1E06348B0
:103C00000078022805D10C2000F0C6F800F015FA63
:103C1000B7E05E480078032840D1FEF7A3FD5C4979
:103C20000968401A5B49884208D257480078C0B2F8
:103C3000C0080100C907C90F00291DD152480078EA
:103C4000C0B2C0080100C907C90F002906D04E48FC
:103C50000078F72101404C48017009E000F070F94C
:103C6000B649086048480078082101434648017079
:103C7000FEF778FD4649086043480078C0B2C008A6
:103C80000100C907C90F002904D0AC48006800F042
:103C9000AAF976E0002000F07FF872E03B48007857
:103CA000042805D10D2000F09EF900F0C6F968E067
:103CB0003648007805285DD1FEF754FD344909687F
:103CC000401A344988421DD32F480078C0B2C0083A
:103CD0000100C907C90F002906D02B480078F72139
:103CE00001402948017009E000F0E7F893490860B5
:103CF000254800780821014323480170FEF732FD72
:103D00002349086020480078C0B2C0080100C907F4
:103D1000C90F002928D0FEF725FD1A490968401A65
:103D2000C8282ED318480078C0B240080100C9073F
:103D3000C90F002909D0002000F02EF812480078A1
:103D4000FD2101401048017009E07C48006800F046
:103D500023F80D480078022101430B480170FEF75B
:103D600001FD084908600CE0FFF704FBC0B200F059
:103D700070F806E0FFF7FEFAC0B200F06AF800F053
:103D80005CF901BD04040020370400203804002041
:103D900008040020B80B000010B50400E00606D4AB
:103DA000002204219020C005FFF729FE05E0012232
:103DB00004219020C005FFF722FEE00706D4002270
:103DC00000219020C005FFF71AFE05E00122002126
:103DD0009020C005FFF713FE200706D40022032120
:103DE0009020C005FFF70BFE05E001220321902083
:103DF000C005FFF704FE600706D4002202219020D0
:103E0000C005FFF7FCFD05E0012202219020C0055E
:103E1000FFF7F5FDA00706D4002201219020C00580
:103E2000FFF7EDFD05E0012201219020C005FFF71D
:103E3000E6FDA00606D4002205219020C005FFF76C
:103E4000DEFD05E0012205219020C005FFF7D7FD2A
:103E500010BD80B50100C9B2002903D10120FFF7D0
:103E60009BFF29E00100C9B2022903D10420FFF71A
:103E700093FF21E00100C9B2012903D10820FFF717
:103E80008BFF19E00100C9B2042903D11020FFF70C
:103E900083FF11E00100C9B2032903D10220FFF71B
:103EA0007BFF09E0C0B2052803D12020FFF774FF93
:103EB00002E01820FFF770FF01BD10B5FEF778FF94
:103EC000002100E0491C202917D2634A1268802390
:103ED0001B069A4209D0604A1268002A05D05E4A41
:103EE000126852005C4B1A6002E001225A4B1A60C1
:103EF000594A12680240002AE4D057480068FEF789
:103F0000BDFF0400202C16D2FEF719FF062804D1AD
:103F1000524804214C4300590EE0FEF710FF0528DB
:103F200004D14F4804214C43005905E04D48042179
:103F30004C43005900E0002010BD00000C0400209C
:103F4000F8B5FEF7FCFE052806D1FEF734FF464A19
:103F5000002302400B4005E0FEF72DFF434A0023FB
:103F600002400B40002400E0641C402C24D2404856
:103F700003C8012680273F06B94208D801D3B042C2
:103F800005D23B4803C8002907D1002805D10120EC
:103F90000021374D03C5083D06E0354803C8001829
:103FA0004941334D03C5083D314803C8104019400D
:103FB000002901D10028D7D02D4803C8FEF7E1FF22
:103FC0000400402C0DD2FEF7BAFE052804D1294882
:103FD00004214C43005905E0274804214C43005973
:103FE00000E00020F2BD10B50400FEF7BBFB234942
:103FF0000968401AC8281FD3FEF7B4FB1F490860A0
:104000001F480078C0B240080100C907C90F002945
:1040100009D01B480078FD2101401948017000209B
:10402000FFF7BAFE08E01648007802210143144861
:1040300001702000FFF7B0FE10BD80B5FEF792FBC7
:1040400010494018104908600D48007808210143C4
:104050000B48017001BD0000C80000203C4800086A
:10406000BC480008BC47000808270600085E820418
:10407000C0000020BC460008BC4500080404002025
:104080003704002048F4FFFF0804002080B500201A
:10409000AA490870FEF766FBA9490860BD48007888
:1040A00001210143BB48017001BD80B5B9480078CA
:1040B0000100C907C90F002928D0A04800780128AD
:1040C00002D100F0FAF823E09C480078022802D1DF
:1040D00000F038F91CE099480078032802D100F07C
:1040E0006AF915E095480078042802D100F070F9CB
:1040F0000EE092480078052802D100F04DF907E063
:1041000000208E49087000F004F801E0FFF7BEFFC0
:1041100001BD80B5FEF726FB89490860FEF748FE21
:10412000002803D00520FFF741FD02E00020FFF743
:104130003DFD98480078FB21014096480170FEF74C
:10414000FEFD042803D1FEF7F7FD172807D2FEF77E
:10415000F6FD062814D1FEF7EFFD142810D3FEF764
:1041600010FE012806D18B480078082101438948B8
:10417000017005E087480078F7210140854801700B
:10418000402000F091F9002806D0824800780821EC
:104190000143804801700AE0402000F089F90028BE
:1041A00005D07C480078F72101407A480170122040
:1041B00000F07AF912280ED1402000F075F900289D
:1041C00009D101205D49087072480078FB21014047
:1041D0007048017070E00C2000F066F90C2809D1DD
:1041E0000220564908706B480078FB21014069485D
:1041F000017061E0032000F057F9032803D1032088
:104200004E49087058E0302000F04EF9302803D1B4
:1042100004204A4908704FE05E480078C0B2C008E8
:104220000100C907C90F002946D1202000F040F93C
:10423000202806D10520FFF7CDF80020FFF7B6FCB7
:104240003AE0012000F034F9012806D10020FFF700
:10425000C1F80020FFF7AAFC2EE0082000F028F9A2
:10426000082806D10120FFF7B5F80020FFF79EFCD3
:1042700022E0022000F01CF9022806D10320FFF7FB
:10428000A9F80020FFF792FC16E0102000F010F9CA
:10429000102806D10420FFF79DF80020FFF786FCC8
:1042A0000AE0042000F004F9042805D10220FFF7F9
:1042B00091F80020FFF77AFC01BD80B5122000F0D4
:1042C000F3F8122836D1FEF74DFA1D490968401A55
:1042D0004649884231D30120FFF768FC2D48007819
:1042E000C0B280080100C907C90F002925D129489B
:1042F0000078C0B2C0080100C907C90F002909D160
:104300002448007808210143224801700120FEF76B
:1043100022FD08E01F480078F72101401D48017088
:104320000020FEF718FD1B480078042101431948BE
:10433000017002E005200149087001BD3A04002027
:104340001004002080B50C2000F0AEF80C281CD121
:10435000FEF708FA26490968401A2649884217D309
:104360000220FFF723FC0B480078C0B28008010050
:10437000C907C90F00290BD1064800780421014361
:1043800004480170FEF707FD02E005201A49087095
:1043900001BD00003904002080B53F2000F084F802
:1043A000002807D13F2000F083F8002802D1002028
:1043B0001149087001BD80B50320FFF7F7FB03200A
:1043C00000F072F8032802D005200B49087001BDE7
:1043D00080B50420FFF7EAFB302000F065F83028B4
:1043E00002D005200449087001BD000088130000B8
:1043F00010040020B80B00003A04002080B5012210
:1044000000216848FFF74CFA01220A216548FFF7AE
:1044100047FA01220B216348FFF742FA01220D21DE
:104420006048FFF73DFA01220E215E48FFF738FA97
:1044300001220F215B48FFF733FA01220621902069
:10444000C005FFF72DFAFEF78DF90A3856490860C6
:1044500001205649087001BD10B554480078012864
:104460001FD153480468FEF77DF94F490968401A87
:104470000A2809D3FEF776F94B49086000F01CF8CA
:1044800000F05EF84A4908604948006860404949C0
:1044900008604848006846490968884345490860FB
:1044A00001E0FFF7ABFF10BD4149096808407047C4
:1044B000404909680840704710B500240021394878
:1044C000FFF7AAFA002802D12000012404430A21A0
:1044D0003448FFF7A1FA002802D120000224044347
:1044E0000B213048FFF798FA002802D1200004245D
:1044F00004430D212B48FFF78FFA002802D120003A
:10450000082404430E212748FFF786FA002802D129
:104510002000102404430F212248FFF77DFA0028D1
:1045200002D120002024044306219020C005FFF77B
:1045300073FA002802D1200040240443200010BD5B
:1045400030B501000A00002006E014001A4A0423D6
:104550004343D2582243401C0328F6D31648C06870
:1045600002400800002306E00500134804245C43D1
:10457000005928405B1C032BF6D310430E4AD06031
:1045800002220AE00C4B042454431B191B1F1B6816
:10459000094C042555436351521E002AF2D1064AA4
:1045A000116030BD000400480004002036040020E3
:1045B000F8030020FC030020D003002000000000CE
:1045C00000000000000000003000000000000000BB
:1045D00000000000000000000000000000000000DB
:1045E00031000000320000003400000037000000FD
:1045F0000000000035000000000000000000000086
:104600003800000000000000000000000000000072
:104610000000000000000000390000000000000061
:10462000000000003A000000000000000000000050
:10463000000000000000000000000000000000007A
:10464000000000000000000000000000000000006A
:10465000000000000000000000000000000000005A
:10466000000000000000000000000000000000004A
:10467000000000000000000000000000000000003A
:10468000000000000000000000000000000000002A
:10469000000000000000000000000000000000001A
:1046A000000000000000000000000000000000000A
:1046B00000000000000000000000000000000000FA
:1046C00000000000000000003000000000000000BA
:1046D00000000000000000000000000031000000A9
:1046E0003200000035000000000000000000000063
:1046F0003800000000000000000000000000000082
:10470000390000003A000000000000000000000036
:104710000000000000000000000000000000000099
:104720000000000000000000000000000000000089
:104730000000000000000000000000000000000079
:104740000000000000000000000000000000000069
:104750000000000000000000000000000000000059
:104760000000000000000000000000000000000049
:104770000000000000000000000000000000000039
:104780000000000000000000000000000000000029
:104790000000000000000000000000000000000019
:1047A0000000000000000000000000000000000009
:1047B00000000000000000000000000001000000F8
:1047C00001000000040000000D00000001000000D6
:1047D0000F000000070000000800000002000000B9
:1047E0000A0000000B0000000B0000001100000098
:1047F000010000000E000000100000000D0000008D
:1048000012000000130000000B0000000D0000006B
:1048100016000000180000001A0000000D00000043
:104820001B0000000D0000001D000000090000003A
:1048300018000000020000001F0000000D00000032
:104840000D000000040000000D0000000100000049
:104850000F000000070000000D0000000200000033
:104860000A0000000B0000000B0000000B0000001D
:104870000B0000000E00000010000000030000000C
:1048800012000000130000000B00000005000000F3
:1048900016000000180000001A00000008000000C8
:1048A0001B0000000D0000001D00000009000000BA
:1048B00018000000020000001F00000001000000BE
:1048C00001000000040000000D00000001000000D5
:1048D000070000000A0000000B0000000B000000B1
:1048E0000E00000010000000120000001300000085
:1048F0000B00000016000000180000001800000067
:104900001A0000001B000000060000000600000066
:104910000600000006000000060000000F00000076
:104920001D0000001D00000011000000020000003A
:104930000D0000000D0000000900000070B401230C
:10494000002413E00168001D194202D04D466D1E7F
:1049500049190C60091D121F042AFAD20D0096078E
:1049600001D50C80AD1C1A4000D02C700268001DCF
:10497000002AE7D170BC704780B5FDF7F6FEFEF760
:10498000ADF9FDF7A1FBFDF752FFFFF737FDFFF78C
:10499000B1F8FFF77BFBFDF71AFFFDF71CFFFFF7F0
:1049A0005BFDFFF782FBFDF7A4FBFFF702F9F4E7DD
:1049B00030B401220168001D00290FD00368C3181C
:1049C00044680830144202D04D466D1E64191D68BB
:1049D00025601B1D241D091FECD0F8E730BC704773
:1049E00010B5074979441831064C7C44163404E06C
:1049F000081D0A68891888470100A142F8D110BD36
:104A0000080000002800000035FFFFFF6C030000D5
:104A1000D00000200000000099FFFFFF1000000000
:104A2000A8000000C00000200000000000F00DF809
:104A3000002801D0FFF7D4FF00BF00BF002000BF57
:104A400000BFFFF799FF00F002F80120704780B522
:104A500000F002F801BDFEE70746384600F002F814
:104A6000FBE7FEE780B500BF00BF024A1100182037
:104A7000ABBEFBE7260002000000000001020304B9
:104A800001020304060708090203040506070809D2
:104A90000A0B0C0D0E0F1010010203040506070887
:104AA000090A0B0C0D0E0F10303132333435363706
:104AB0003839414243444546014880470148004750
:104AC000DF270008D94A00080100000000000000AC
:104AD0000100000000127A0000BF00BF00BF00BF4D
:104AE000FFF7A4FFFEE7FEE7FEE7FEE7FEE7FEE7CF
:104AF000FEE7FEE7FEE7FEE7FEE7FEE7FEE7FEE78E
:084B0000FEE7FEE7FEE7FFFF00
:0400000508004AD9CC
:00000001FF
